:10000000B2018E2AA501A400B3172730A300103037
:1000100015200330A300E8301520A301643015201B
:10002000A3010A30152024082028A2002508A100D9
:100030002408A0004C222008031DB313B31B0800A2
:10004000303E23280408A20083168612831209304A
:10005000A30003103220A20CA30B2A280314322081
:100060000314892A031837280000861239288616B7
:1000700039280030A1006230F829B216B21EB2123F
:10008000B2194628B2157F2003186D280830A30046
:100090009320A20DA30B4828B21E78209D20992002
:1000A000B21A6D20722022080310892AB216B21EDD
:1000B000B21232196028FE39B30032150310892AB2
:1000C000321A6828A60032167F2003186D282608E9
:1000D000862003186D28B21E892A78209D203211AF
:1000E0003212B211360884003408841780047E2846
:1000F00036088400340980058417800508007220C2
:100100009D20782099203308B2190138A2000830C8
:10011000A300A20D03187220031C78209D209920B3
:10012000A30B892872209D2036088400340800051E
:10013000FF3E3708840035097B28370884003508DE
:100140007528083033190130A300A2013608840055
:100150003408C221340880048922892284130005CE
:10016000FF3E331DA20C3319A20D3230F721A30B31
:10017000A82822080314892AA20008303319013064
:10018000A300A20C360884003408C22134080318E6
:1001900080043730F72134088004A30BC1280314EE
:1001A000892AB31C892AD728B300331C892A360828
:1001B00084003408C2210130A100E030F821340865
:1001C00080040130A100E030F829B40084178004D5
:1001D0008413A201201CA20007210319892A0721E8
:1001E0000319892A0721892AB400C521200821047E
:1001F0000319892A7E2284133408800664000029AA
:100200000129A00A0319A10FFE288006892A3408B3
:10021000A2060130A000A101000834052206031D3A
:100220000800A00A0319A10F0C2908003708A00034
:100230003508A1000130A200A30164003E21031C87
:100240003129A20B1D29FF30A30703181D29A00780
:10025000031CA107031C08006430A2000030A300A7
:100260001D296F210830A30070213E21A20C3829DE
:10027000A30B3429702103142208080036088400D7
:100280003408841780048413000533193406FF3EB4
:100290000800A600360884000930A7000310552185
:1002A000A60CA70B4F29031455298413B31D6429E9
:1002B00000083404331D3406800084170008340419
:1002C000031C34068000702900083404031C340623
:1002D00033193406800084173409800570293317D8
:1002E00001308A00330D0639A0008221A1000130BF
:1002F0008A00200A8221331FF8293313A00002301C
:100300001922F829863E03188A0A820001348B34A8
:1003100003342B34003452340C34EF34A400290855
:100320000319892A8422A000251883172408840031
:10033000200880008313A40AA9038F29B313290876
:100340000319B3170430A800250EAB212508AB21F3
:10035000240EAB2124080F39F63E0318073E0A3E4F
:10036000B129A000A8030319B31329080319BB2955
:100370002802031808002008031DB313B31B08004C
:10038000303E842AFF3A8005C629FF3A841780054B
:10039000892A83178001840AFF3E031DCA29892AFE
:1003A000031783168C010C1483120C0803178D0A93
:1003B000892A030103178C0083168C010C15553014
:1003C0008D00AA308D008C148C18E4290C11831236
:1003D0008D0A892AA301A200FF30A207031CA307EC
:1003E000031C892A0330A100E330F821EC29A10184
:1003F000F43EA000A109FE30031C012AA007031847
:10040000FE29A0076400A10FFE2900002018082A79
:1004100020180A2A08002E220E2A28220319142A3C
:100420002308A1002208A000200808000310A10C46
:10043000A00CFF3E0318162A2008892AA2000230C9
:10044000312AA101A301A2000330312AA101A30195
:10045000A2000130312AA2000630312AA200043065
:10046000312AA80023082102031D382A220820026D
:10047000043003180130031902302805031DFF3032
:10048000892A0038031DFF300405031DFF30892A27
:100490000404031DFF30892AA501A4011030A60021
:1004A000210DA40DA50D2208A4022308031C230F6F
:1004B000A5020318622A2208A40723080318230FA1
:1004C000A5070310A00DA10DA60B502A2008892A0C
:1004D0001030A800A101A001A70CA60C031C762ACD
:1004E0002208A00723080318230FA107A10CA00CC2
:1004F000A50CA40CA80B6C2A2408892AA009A10920
:10050000A00A0319A10A0800840031088A003008F3
:10051000820083130313831264000800C0309F001D
:10052000831675308F008312031787018801031328
:10053000393090008316FF30850086019F30870098
:1005400003170F30880089018312031341309F0085
:10055000831680309F0083122030840060308A012F
:10056000CA21A030840050308A01CA211030840092
:1005700060308A01C9219030840060308A01C9212D
:1005800020308600871207130317FC308D000313F9
:100590008A01D021D2000317FD308D0003138A0198
:1005A000D021D3000317FE308D0003138A01D02120
:1005B000E2000317FF308D0003138A01D021E3000E
:1005C0000317FA308D0003138A01D021C8000317E6
:1005D000FB308D0003138A01D021C9000317F830C6
:1005E0008D0003138A01D021DA000317F9308D0042
:1005F00003138A01D021DB000317F4308D000313AD
:1006000052088A01DA210317F5308D0003135308CD
:100610008A01DA210317F6308D0003135A088A0184
:10062000DA210317F7308D0003135B088A01DA2102
:100630000730B6000430B40001308A01D4205530B0
:100640008A01BC2028308A01BC20B9308A01BC2034
:1006500011308A01BC2016308A01BC2001308A0189
:10066000BC2000308A01BC2000308A01BC20A430AC
:100670008A01BC2044308A01BC208A01D120073085
:10068000B6000430B40001308A01D42055308A010C
:10069000BC2028308A01BC20D6308A01BC202D30F5
:1006A0008A01BC2016308A01BC2001308A01BC209E
:1006B00000308A01BC2000308A01BC20E6308A016B
:1006C000BC2044308A01BC208A01D1200614831644
:1006D000061083120330A300E8308A01EB210610D4
:1006E000831606101B3083128A01232046308A01AC
:1006F00023201B308A0123202E308A0123201B3027
:100700008A01232043308A01232042308A0123209A
:100710004D308A01232053308A01232020308A0162
:1007200023204D308A01232061308A012320733039
:100730008A01232074308A01232065308A01232016
:1007400072308A01232020308A01232056308A010A
:10075000232030308A0123202E308A01232030309C
:100760008A01232038308A01232042308A01232045
:1007700079308A01232020308A01232050308A01D9
:10078000232065308A01232074308A0123206530BC
:100790008A01232072308A01232020308A012320FD
:1007A00050308A01232065308A01232072308A016B
:1007B00023206B308A01232069308A0123206E3088
:1007C0008A01232073308A01232077308A01232075
:1007D00077308A01232077308A0123202E308A0146
:1007E000232031308A01232035308A012320303004
:1007F0008A0123206D308A01232070308A01232052
:1008000067308A0123202E308A01232063308A0139
:1008100023206F308A0123202E308A012320753057
:100820008A0123206B308A0123200A308A01232089
:100830000D308A01232038308A0123206D308A014F
:10084000232068308A0123207A308A012320203037
:100850008A01232028308A01232001308A010220C6
:1008600029308A01232020308A01232043308A0145
:10087000232065308A0123206C308A0123206C30CC
:100880008A01232073308A01232021308A0123200A
:100890000730A300D0308A01EB211B308A012320CE
:1008A00043308A012320DB30D6000B30D7005608B6
:1008B0008E0057088F000C100830860683168611AC
:1008C00083128A110A12F4248A150A12A9218A15A0
:1008D0000A1258208A150A12A2238A150A122D27F5
:1008E00064006908043C8A110A12031D7A2C8A15D7
:1008F0000A12CE276400013070028A110A12031C0A
:10090000852CF10A8A110A12862CF1018A110A1625
:1009100092227108A00002308A012122DC007008B6
:10092000A00000308A012622DE005C0884005E08F8
:100930008A014122DE00DF0064005E085F048A1144
:100940000A120319A62C8A150A125A25F001FA0A6E
:1009500064007A08283C8A110A12031DE82C031748
:10096000FC308D00031352088A01DA210317FD3091
:100970008D00031353088A01DA210317FE308D001E
:10098000031362088A01DA210317FF308D00031375
:1009900063088A01DA210317FA308D00031348082F
:1009A0008A01DA210317FB308D00031349088A01FD
:1009B000DA210317F8308D0003135A088A01DA216F
:1009C0000317F9308D0003135B088A01DA21FA015D
:1009D00064008A110A120C1CE82C56088E00570875
:1009E0008F000C108A015C2C06158316061103304B
:1009F00083128A01EA21061183160611013083123F
:100A00008A01EA212830A000A101063084000430C8
:100A10008A01F420FF30E600E701D401D50132302D
:100A20008A01EA21061583160611033083128A0112
:100A3000EA21061183160611013083128A01EA2188
:100A40001430A000A1010630840004308A01F42093
:100A50000130E4006400023064028A110A120318B3
:100A6000892DC201C3010730B6008030B4000630C2
:100A7000B3006430B700B5018A0116218A110A1249
:100A8000031C892FC2006400420867028A110A12FF
:100A900003184E2D4208E7006408F700640066085A
:100AA00042028A110A120318592D4208E60064080E
:100AB000F800AF30C2070318C30A4208A000430879
:100AC000A1000130A3007C308A012B228A110A1276
:100AD000031D6E2D0130F0006408F6004208A000EE
:100AE0004308A100A301DC308A0123228A110A12E3
:100AF000031D7E2D0230F0006408F6004208D40782
:100B000043080318013ED507E40A8A110A12031D9F
:100B10002A2D061583160611033083128A01EA2155
:100B2000061183160611013083128A01EA213C3036
:100B3000A000A1010630840004308A01F420640082
:100B40007408013C8A110A12031DCE2D5408A0001E
:100B50005508A1004F08A3004E088A0123228A11DC
:100B60000A12031DCA2D5408CE025508031C013E6B
:100B7000CF024E08A0004F08A100A30132308A0125
:100B80002B228A110A12031DC72D0630F0008A118C
:100B90000A12CE2D5408CE005508CF005408A000EC
:100BA0005508A1006430A200A3018A014C22E40090
:100BB0002108E5005408A0005508A1006430A200F7
:100BC000A3018A014C222408DC002508DD005C0812
:100BD000A0005D08A1000A30A200A3018A014C22F6
:100BE000E8002108E9006408FF001B308A01232087
:100BF00053308A01232000308A01232000308A01EB
:100C0000232056308A0123206F308A0123206C3044
:100C10008A01232020308A0123206508A50064086A
:100C20008A0103202E308A0123206908A500680864
:100C30008A01032020308A01232056308A01232094
:100C400020308A012320AF306707E400E501E50D7D
:100C50006408A0006508A1000130A3006D308A017E
:100C60002B228A110A12031D402E86148316861029
:100C7000831207178316071383128A110A12442E50
:100C800007138316071383126408A0006508A100E8
:100C90006430A200A3018A014C22E8002108E90087
:100CA0006408A0006508A1006430A200A3018A01C5
:100CB0004C222408EA002508EB007708E4001B30EA
:100CC0008A01232053308A01232000308A01232007
:100CD00001308A01232048308A01232069308A01AB
:100CE000232056308A01232020308A0123205B30C4
:100CF0008A01232064000A3064028A110A12031850
:100D0000842E30308A0123206A08A0006B08A100DD
:100D1000A3010A308A0123228A110A12031DB52E6B
:100D200064088A0102205D308A01232020308A0174
:100D300023206908A50068088A0103202E308A0153
:100D4000232030308A0123206B08A5006A088A011D
:100D5000032020308A01232056308A0123202030AE
:100D60008A0123208A110A12D42E64088A010220E3
:100D70005D308A01232020308A0123206908A500E4
:100D800068088A0103202E308A0123206B08A50001
:100D90006A088A01032020308A01232056308A0104
:100DA000232020308A012320AF306607E400E501CC
:100DB000E50D6408A0006508A100A301E6308A01E2
:100DC00023228A110A12031DF02E0616831606121C
:100DD000831287168316871283128A110A12F82E3D
:100DE0000612831606128312871283168712831245
:100DF0006408A0006508A1006430A200A3018A0174
:100E00004C22E8002108E9006408A0006508A10060
:100E10006430A200A3018A014C222408EA002508BC
:100E2000EB007808E4001B308A01232053308A014C
:100E3000232000308A01232002308A0123204C30F5
:100E40008A0123206F308A01232056308A01232013
:100E500020308A0123205B308A01232064000A307D
:100E600064028A110A120318382F30308A012320B5
:100E70006A08A0006B08A100A3010A308A0123229E
:100E80008A110A12031D692F64088A0102205D304D
:100E90008A01232020308A0123206908A5006808E0
:100EA0008A0103202E308A01232030308A0123203A
:100EB0006B08A5006A088A01032020308A012320DC
:100EC00056308A01232020308A0123208A110A12F9
:100ED000882F64088A0102205D308A012320203097
:100EE0008A0123206908A50068088A0103202E30A2
:100EF0008A0123206B08A5006A088A01032020309C
:100F00008A01232056308A01232020308A012320A1
:100F100008006408F6000330F0000800E601E7016D
:100F2000E401E50149309F000130E90064000B3025
:100F300069028A110A120318B62F9F1464008A11DD
:100F40000A129F1CA52F8A019E2F1E08EB008316F4
:100F50001E088312EA006A08E4076B080318013EC2
:100F6000E507E90A8A110A12031D962F4D309F00EA
:100F70000130E90064000B3069028A110A1203187B
:100F8000DA2F9F1464008A110A129F1CC92F8A014C
:100F9000C22F1E08ED0083161E088312EC006C0899
:100FA000E6076D080318013EE707E90A8A110A12ED
:100FB000031DBA2F6608A0006708A1000A30A2002E
:100FC000A3018A014C22E6002108E7006408A00082
:100FD0006508A1000A30A200A3018A014C22E400A6
:100FE0002108E50030306402DC000230031C013EC1
:100FF0006502DD005D0C5C0CFC0030306602DC003C
:101000000230031C013E6702DD005D0C5C0CFD003C
:101010007C08A00032308A012622DC007D08A00076
:1010200032308A012622DE005C0884005E088A01D4
:101030004822DE00DF0064005E085F048A150A12A1
:10104000031924280430F0001B308A012320533078
:101050008A01232000308A01232003308A012320C3
:1010600054308A01232065308A0123206D308A01A3
:10107000232020308A01232046308A01232064085F
:101080008A01022020308A01232052308A01232045
:1010900066088A01022020308A012320F8308A0164
:1010A000232043308A01232020308A012320080096
:1010B0001B308A01232053308A01232000308A010B
:1010C000232003308A01232054308A0123206530F5
:1010D0008A0123206D308A01232020308A012320B9
:1010E0000730B6000430B40001308A01D4205530F6
:1010F0008A01BC2028308A01BC20D6308A01BC205D
:101100002D308A01BC2016308A01BC2001308A01B2
:10111000BC2000308A01BC2000308A01BC20E630AF
:101120008A01BC20BE308A01BC208A01D1208A15E8
:101130000A124D211B308A01232053308A012320BB
:1011400000308A01232003308A01232054308A0191
:10115000232065308A0123206D308A01232020302E
:101160008A01232066088A0123206A088A01022056
:101170002E308A0123206B088A01022020308A0148
:1011800023200730B6000430B40001308A01D42097
:1011900055308A01BC2028308A01BC20D6308A0113
:1011A000BC202D308A01BC2016308A01BC200130C1
:1011B0008A01BC2000308A01BC2000308A01BC209A
:1011C000E6308A01BC2044308A01BC208A01D1204B
:1011D0006A08FC000730B6000430B40001308A0110
:1011E000D42055308A01BC2028308A01BC20B93077
:1011F0008A01BC2011308A01BC2016308A01BC2033
:1012000001308A01BC2000308A01BC2000308A01F4
:10121000BC20A4308A01BC20BE308A01BC208A01D7
:10122000D1208A150A124D2166088A0123206A08F6
:101230008A0102202E308A0123206B088A010220B5
:1012400020308A0123200730B6000430B40001307A
:101250008A01D42055308A01BC2028308A01BC2064
:10126000B9308A01BC2011308A01BC2016308A01B5
:10127000BC2001308A01BC2000308A01BC20003033
:101280008A01BC20A4308A01BC2044308A01BC20E1
:101290008A01D1206A08FD0008000730B60004303A
:1012A000B40002308A01D4208A01A120E4008A011E
:1012B000A120E5008A01D1202B30E6006408A000BF
:1012C0006508A100FC30A3008F308A012B228A150B
:1012D0000A12031D72292D30E600E509E409E40A2B
:1012E0000319E50A6408A6006508A7000530A200F6
:1012F000A3018A016822DC002508DD005C08A0004B
:101300005D08A1000830A200A3018A014C22E4007C
:101310002108E5006408A0006508A1000A30A200C9
:10132000A3018A014C22EA006408A0006508A1001C
:101330000A30A200A3018A014C222408EB006400B9
:1013400033306A028A150A12031CA8290430F000FF
:101350000800E601E70141309F000130E50064002C
:101360000B3065028A150A120318D0299F146400F5
:101370008A150A129F1CBF298A150A12B7291E084E
:10138000C10083161E088312C0004008E60741080A
:101390000318013EE707E50A8A150A12031DAF2963
:1013A0006608A0006708A1000A30A200A3018A0114
:1013B0004C22C0002108C1004008A0004108A10043
:1013C0000130A300FB308A0123228A150A12031D73
:1013D0000D2A4008FE3CDC004108031C013E013C94
:1013E000DD000330A000A101A30163308A010D22BA
:1013F000DE002108DF005C08A0005D08A1005E0897
:10140000A2005F08A3008A014C22C0002108C1008D
:101410002B30F3008A150A12422A4008A000410826
:10142000A1000230A30000308A012B228A150A1283
:10143000031D3E2A00304002DC000230031C013E46
:101440004102DD000330A000A101A30163308A0145
:101450000D22DE002108DF005C08A0005D08A1006D
:101460005E08A2005F08A3008A014C22C000210888
:10147000C1002D30F3008A150A12422AC001C101B1
:101480003D30F3005408A0005508A1006430A200CC
:10149000A3018A014C22DC002108DD005C08A600C3
:1014A0005D08A7004008A2004108A3008A01682245
:1014B000E4002508E5006408A0006508A100E83004
:1014C000A2000330A3008A014C222408DC00250876
:1014D000DD005C08A0005D08A1006430A200A3014B
:1014E0008A014C22E6002108E7006408A000650894
:1014F000A100E830A2000330A3008A014C22E400DE
:101500002108E5001B308A01232053308A01232063
:1015100000308A01232004308A01232041308A01CF
:1015200023206D308A01232070308A01232020304F
:101530008A01232073088A0123204108A50040085E
:101540008A01032020308A0123204B308A01232086
:1015500020308A0123206508A50064088A01032041
:101560002E308A0123206708A50066088A0103201F
:1015700020308A0123204008A6004108A7006430DB
:10158000A200A3018A016822DC002508DD005C08B6
:10159000A0005D08A1002430A200A3018A014C2212
:1015A000C0002108C100640073082B3C8A150A1290
:1015B000031D062B4008C40741080318013EC50758
:1015C0004408A0004508A100A30114308A012E227E
:1015D0008A150A12031D062B0130A000A1013A3022
:1015E000A30098308A010D22DC002108DD005C0890
:1015F000DA075D080318013EDB071430C40200302F
:10160000031C013EC5028A150A12E02A6400730811
:101610002D3C8A150A12031D382B4008C6074108C5
:101620000318013EC7074608A0004708A100A30110
:1016300014308A012E228A150A12031D382B01301C
:10164000A000A101A30101308A010B22DC002108C6
:10165000DD005C08DA025D08031C013EDB02143089
:10166000C6020030031C013EC7028A150A12132B62
:101670005A08A0005B08A1006430A200A3018A01FF
:101680004C22E8002108E9006808FB005A08A00085
:101690005B08A1006430A200A3018A014C22240847
:1016A000E4002508E5001B308A01232053308A011D
:1016B000232000308A01232005308A012320533063
:1016C0008A0123206F308A01232063308A0123207E
:1016D00020308A0123206908A50068088A010320B8
:1016E0002E308A0123206408A0006508A100A30110
:1016F0000A308A0123228A150A12031D932B3030E7
:101700008A0123206508A50064088A01032020308F
:101710008A01232025308A01232020308A012320BA
:101720008A150A12A12B6508A50064088A01032006
:1017300020308A01232025308A01232020308A018D
:10174000232008000130A0000730840002308A0105
:10175000E5202008E6002108E7006608A0006708E9
:10176000A100A30100308A011E228A150A12031D5E
:10177000D92B6608A0006708A1000B30A200A301C6
:101780008A014C22E6002108E700E430A0001E3068
:10179000A1006608A2006708A3008A014C22DC00B1
:1017A0002108DD0001305C07E6005D080318013EFA
:1017B000E7001B308A01232053308A0123200030A8
:1017C0008A01232006308A0123204D308A012320FC
:1017D00070308A01232068308A01232020308A015A
:1017E00023206708A50066088A01032020308A01AB
:1017F000232077308A01232068308A0123202F306C
:101800008A0123206D308A01232020308A01232081
:101810006F08A5006E088A01032020308A0123206A
:1018200020308A0123206608A6006708A7009230AE
:10183000A200A3018A016822E6002508E7006608E5
:10184000C80767080318013EC9074808A0004908EF
:10185000A100CE30A30040308A012E228A150A1240
:10186000031DD22CFE0A0130A000A1012730A300E5
:101870000F308A010D22DC002108DD005C08E20740
:101880005D080318013EE307640064080A3C8A15FA
:101890000A12031DC92CD20A0319D30A0317F43004
:1018A0008D0003138A01D021E4000317F5308D0069
:1018B00003138A01D021E5000317F6308D000313CE
:1018C0008A01D021E8000317F7308D0003138A0145
:1018D000D021E90064085202E4006508031C013EBF
:1018E0005302E5005A086802E6005B08031C013E4B
:1018F0006902E7006608A0006708A1006408A2006A
:101900006508A3008A014C22E8002108E9005A0872
:10191000A0005B08A1006808A2006908A3008A0172
:101920004C22EA002108EB006A08CA006B08CB00D1
:101930006808A6006908A7000430A200A3018A0174
:101940006822DC002508DD005C08A6005D08A70011
:101950001030A200A3018A016822DC002508DD0006
:101960006430A000A1010330A300E7308A010D22FA
:10197000DE002108DF005C08A0005D08A1005E0811
:10198000A2005F08A3008A014C22EE002108EF00AC
:10199000FE014030C802CE30031C013EC9028A1548
:1019A0000A12252C1B308A01232053308A01232060
:1019B00000308A01232007308A0123204F308A011A
:1019C000232064308A0123206F308A0123202030B5
:1019D0008A0123205308A50052088A0103202030E1
:1019E0008A01232052308A01232065308A01232076
:1019F0006D308A01232020308A0123204B08A50066
:101A00004A088A01032020308A0123206208A000AE
:101A10006308A1000A30A200A3018A014C22E4005D
:101A20002108E5006208A0006308A1000A30A200B6
:101A3000A3018A014C222408E6002508E7001B3098
:101A40008A01232053308A01232000308A01232079
:101A500008308A01232054308A01232072308A0101
:101A6000232069308A01232020308A012320650841
:101A7000A50064088A0103202E308A01232067080C
:101A8000A50066088A01032020308A012320433004
:101A90008A01232068308A01232067308A012320AD
:101AA00020308A01232074088A01022020308A0114
:101AB000232008001B308A0123205E308A01232066
:101AC00064308A01EA211B308A01232021308A01F7
:101AD00023201B308A01232043308A012320203019
:101AE0008A0123202A308A01232020308A012320E2
:101AF00042308A0123204D308A01232053308A014D
:101B0000232020308A01232041308A0123206C3099
:101B10008A01232061308A01232072308A01232028
:101B20006D308A01232073308A01232020308A01FE
:101B300023202A308A01232020308A0123200A30E2
:101B40008A0123200D308A012320061483160610F3
:101B500083128614831686108312061683160612C5
:101B600083120613831606138312F40164007008AF
:101B7000013C8A150A12031DE72D43308A012320F8
:101B800065308A0123206C308A0123206C308A0161
:101B9000232020308A01232076088A010220203069
:101BA0008A0123203E308A01232041308A012320EC
:101BB0004D308A01232061308A01232078308A0148
:101BC000232056308A01232020308A0123206400FC
:101BD0007008023C8A150A12031D182E43308A0130
:101BE000232065308A0123206C308A0123206C3049
:101BF0008A01232020308A01232076088A010220CE
:101C000020308A0123203C308A01232041308A0180
:101C100023204D308A01232069308A0123206E3031
:101C20008A01232056308A01232020308A01232074
:101C300064007008033C8A150A12031D462E4330C7
:101C40008A01232065308A0123206C308A012320F9
:101C50006C308A01232020308A01232076088A01F3
:101C6000022020308A01232045308A01232072304F
:101C70008A01232072308A0123206F308A012320B9
:101C800072308A01232021308A01232064007008E9
:101C9000043C8A150A12031D7D2E50308A01232030
:101CA00061308A01232063308A0123206B308A014E
:101CB00023203E308A01232041308A0123206230D4
:101CC0008A01232073308A0123204D308A0123208A
:101CD00061308A01232078308A01232054308A0120
:101CE000232065308A0123206D308A012320703043
:101CF0008A01232020308A01232064007008053CDB
:101D00008A150A12031DB42E20308A0123202030A8
:101D10008A01232041308A0123206C308A0123204C
:101D200061308A01232072308A0123206D308A01BC
:101D3000232020308A01232054308A01232065305B
:101D40008A01232073308A01232074308A012320E2
:101D500021308A01232020308A01232020308A016B
:101D6000232020308A01232064007008063C8A1555
:101D70000A12031D1B2F20308A01232020308A01E4
:101D8000232043308A01232068308A0123206130D8
:101D90008A01232072308A01232067308A012320A0
:101DA00065308A01232020308A01232045308A01B2
:101DB00023206E308A01232064308A0123202130C1
:101DC0008A01232020308A01232020308A01232009
:101DD00020308A01232020308A01232056308A01B6
:101DE00023206F308A0123206C308A012320743035
:101DF0008A01232061308A01232067308A01232051
:101E000065308A01232020308A01232044308A0152
:101E1000232072308A0123206F308A012320703002
:101E20008A01232020308A01232020308A012320A8
:101E300020308A012320F001F1010730A300D030C7
:101E40008A01EB210610831606101B3083128A01CB
:101E500023205F308A012320080045309F000A308C
:101E60008A01EA219F1464008A150A129F1C3B2FE5
:101E70008A150A12332F1E08EB0083161E088312E0
:101E8000EA006A08A0006B08A1000430A200A301C8
:101E90008A014C22EA002108EB000630EA07031809
:101EA000EB0A6A08A0006B08A1002A30A200A30177
:101EB0008A014C22EA002108EB000130EA020030DE
:101EC000031C013EEB026A08E9000800E201E3019D
:101ED0000317FE308D00031362088A01DA2103170D
:101EE000FF308D00031363088A01DA218A110A1674
:101EF0003129D201D3010317FC308D00031352089E
:101F00008A01DA210317FD308D00031353088A017B
:101F1000DA218A110A1631290530F0000800103044
:101F2000DA002730DB000317F8308D0003135A085E
:101F30008A01DA210317F9308D0003135B088A0147
:101F4000DA218A110A1631296400013070028A15DB
:101F50000A12031CAC2F080064007408003C8A15A8
:101F60000A12031DC62F0130F40086108316861056
:101F7000831206128316061283120617831606139F
:101F80008312CE01CF018A150A12CB2FF40106135A
:101F90008316061383128A110A1631291B308A010F
:101FA00023205E308A01232064308A01EA211B301D
:101FB0008A01232043308A0123202A308A012320EA
:101FC00020308A01232020308A01232053308A01C7
:101FD000232075308A01232062308A01232020309B
:101FE0008A0123204D308A01232065308A01232075
:101FF0006E308A01232075308A01232020308A0127
:10200000232031308A01232020308A0123202030F0
:102010008A0123202A308A0123200A308A012320C2
:102020000D308A01232053308A01232074308A0125
:10203000232061308A01232072308A0123207430EA
:102040008A01232020308A01232043308A01232063
:1020500068308A01232061308A01232072308A018E
:10206000232067308A01232065308A012320203015
:102070008A0123203D308A01232020308A01232039
:1020800055308A01232052308A01232065308A018D
:10209000232073308A01232065308A012320743085
:1020A0008A01232020308A01232053308A012320F3
:1020B0006F308A01232063308A01232020308A0177
:1020C000232020308A01232020308A012320203041
:1020D0008A0123203D308A01232020308A012320D9
:1020E0004C308A01232052308A01232065308A0136
:1020F000232073308A01232065308A012320743025
:102100008A01232020308A01232054308A01232091
:1021100072308A01232069308A01232070308A01BD
:10212000232020308A01232020308A0123202030E0
:102130008A0123203D308A01232020308A01232078
:1021400044308A01232052308A01232065308A01DD
:10215000232073308A01232065308A0123207430C4
:102160008A01232020308A0123204F308A01232036
:1021700064308A0123206F308A01232020308A01B5
:10218000232020308A01232020308A012320203080
:102190008A0123203D308A01232020308A01232018
:1021A00052308A01232053308A01232075308A015E
:1021B000232062308A01232020308A0123204D30E1
:1021C0008A01232065308A0123206E308A01232072
:1021D00075308A01232020308A01232032308A0181
:1021E000232020308A01232020308A012320203020
:1021F0008A0123203D308A01232020308A012320B8
:1022000043308A0123200730A300D0308A01EB211C
:102210008A150A122D2764006908003C8A150A12E3
:102220000319A42F64006908013C8A150A120319D6
:102230008F2F64006908023C8A150A120319662F61
:1022400064006908033C8A150A120319792F640097
:102250006908043C8A110A16031938298A110A16DA
:1022600008291B308A0123205F308A0123200800BF
:102270001B308A01232043308A0123202A308A011F
:10228000232020308A01232020308A01232053304C
:102290008A01232075308A01232062308A0123209D
:1022A00020308A0123204D308A01232065308A01A5
:1022B00023206E308A01232075308A0123202030AC
:1022C0008A01232032308A01232020308A012320F2
:1022D00020308A0123202A308A0123200A308A01F3
:1022E00023200D308A01232043308A0123206530CA
:1022F0008A0123206C308A0123206C308A0123203C
:1023000020308A01232056308A0123206F308A0131
:1023100023206C308A01232074308A01232061300D
:102320008A01232067308A01232065308A01232017
:1023300020308A0123203D308A01232020308A0169
:10234000232055308A01232053308A0123206C300A
:102350008A01232061308A01232076308A012320DC
:1023600065308A01232020308A01232055308A01DC
:10237000232070308A01232064308A0123206130B9
:102380008A01232074308A01232065308A012320AA
:1023900020308A0123203D308A01232020308A0109
:1023A00023204C308A01232054308A0123207830A6
:1023B0008A01232020308A01232042308A012320F1
:1023C0004D308A01232053308A01232020308A0196
:1023D000232044308A01232061308A012320743075
:1023E0008A01232061308A01232020308A012320A2
:1023F00020308A0123203D308A01232020308A01A9
:10240000232044308A01232054308A012320653060
:102410008A0123206D308A01232070308A01232015
:1024200020308A01232052308A0123206F308A0114
:1024300023206D308A01232020308A012320203080
:102440008A01232020308A01232020308A01232082
:1024500020308A0123203D308A01232020308A0148
:10246000232052308A01232045308A0123207830EE
:102470008A01232069308A01232074308A012320B5
:1024800020308A01232020308A01232020308A0135
:10249000232020308A01232020308A01232020306D
:1024A0008A01232020308A01232020308A01232022
:1024B00020308A0123203D308A01232020308A01E8
:1024C000232043308A0123200730A300D0308A0123
:1024D000EB218A150A122D2764006908003C8A1135
:1024E0000A160319B52B64006908013C8A110A1603
:1024F0000319EE2C64006908023C8A110A160319BC
:10250000F12A64006908033C8A150A160319762823
:1025100064006908043C8A110A16031931298A11DA
:102520000A16692A0730B6001030B4000730B70029
:102530000830B500A0308A01582051088A0158207F
:1025400050088A01582070088A015620D00A0319C1
:10255000D10A0630B6008030B4000430B3005530E4
:102560008A01492155308A01492155308A01492182
:1025700055308A01492155308A0149210A308A01A2
:10258000EA210630B6008030B4000430B300623077
:102590008A0149216D308A01492173308A0149211C
:1025A00000308A01492170088A01492176088A0190
:1025B00049210730B6001030B4000730B7000830AA
:1025C000B500A0308A01582051088A0158205008CF
:1025D0008A01582076088A015620D00A0319D10AA8
:1025E00008001B308A01232043308A012320543005
:1025F0008A01232078308A01232064308A01232035
:1026000020308A0123205108A50050088A010320A8
:1026100020308A01232042308A01232079308A0128
:10262000232074308A01232065308A0123207330EF
:102630008A0123200A308A0123200A308A012320BC
:102640000D308A01232042308A01232065308A011F
:10265000232020308A01232050308A01232061303A
:102660008A01232074308A01232069308A012320C3
:1026700065308A0123206E308A01232074308A015C
:10268000232021308A0123200630B6008030B40098
:102690000430B30055308A01492155308A0149215F
:1026A00055308A01492155308A01492155308A0126
:1026B000492105308A01EA210630B6008030B40095
:1026C0000430B30062308A0149216D308A0149210A
:1026D00073308A01492101308A01492105308A017C
:1026E000EA21E401E5016408A0006508A1005108A1
:1026F000A30050088A0128228A110A16031DA92B5B
:102700000730B6001030B4000730B7000830B5000D
:10271000A0308A01582051088A01582050088A01A7
:1027200058208A013D20E6000630B6008030B40013
:102730000430B30066088A014921083086068316F2
:1027400086118312E40A0319E50A8A110A16031D89
:10275000732B0630B6008030B4000430B300FF3075
:102760008A0149218A110A16EC2F1B308A01232085
:1027700043308A0123200130E50006158316061137
:10278000033083128A01EA210611831606110130F3
:1027900083128A01EA211430A000A10106308400CE
:1027A00004308A01F4200130E40064000230640245
:1027B0008A110A160318FA2BC201C3010730B600AA
:1027C0008030B4000630B3006430B700B5018A0130
:1027D00016218A110A12031C892FC20064006408A2
:1027E00065028A110A160319FA2BE40A8A110A16DD
:1027F000031DD52BAF30C2070318C30A4208A0003F
:102800004308A1006430A200A3018A014C22E60023
:102810002108E7004208A0004308A1006430A2009C
:10282000A3018A014C222408E8002508E900680871
:10283000A0006908A100A3010A308A0123228A119D
:102840000A16031D5A2C43308A01232065308A0161
:1028500023206C308A0123206C308A012320203011
:102860008A01232065088A01022020308A01232062
:1028700020308A0123206708A50066088A0103200A
:102880002E308A01232030308A0123206908A500D8
:1028900068088A01032056308A01232020308A01EB
:1028A00023200A308A0123200D308A0123208A1137
:1028B0000A168B2C43308A01232065308A0123209D
:1028C0006C308A0123206C308A01232020308A0159
:1028D000232065088A01022020308A01232020302D
:1028E0008A0123206708A50066088A0103202E308C
:1028F0008A0123206908A50068088A010320563050
:102900008A01232020308A0123200A308A012320D3
:102910000D308A0123208A150A122D2764006908C8
:10292000023C8A110A16031D8B2CE50A6400013053
:1029300065028A110A16031CBD2B0130A300F43076
:102940008A01EB210A308A0123200D308A012320DD
:1029500041308A0123206E308A01232079308A0198
:10296000232020308A0123204B308A012320653028
:102970008A01232079308A01232020308A012320F4
:1029800054308A0123206F308A01232020308A01AD
:10299000232045308A01232078308A0123206930A2
:1029A0008A01232074308A01232021308A012320C8
:1029B0000330A300E8308A01EB218A150A122D2783
:1029C00064006908053C8A110A160319DD2C1B30C6
:1029D0008A0123205F308A01232008000930E800A3
:1029E0001B308A01232043308A0123202A308A01A8
:1029F000232020308A01232053308A0123206C3089
:102A00008A01232061308A01232076308A01232025
:102A100065308A01232020308A01232055308A0125
:102A2000232070308A01232064308A012320613002
:102A30008A01232074308A01232065308A012320F3
:102A400020308A0123202A308A01232020308A0165
:102A5000232055308A01232073308A0123206530DA
:102A60008A01232020308A01232055308A01232027
:102A700070308A0123202F308A01232044308A01BC
:102A800023206F308A01232077308A0123206E3083
:102A90008A01232020308A01232074308A012320D8
:102AA0006F308A01232020308A01232020308A01C0
:102AB000232053308A01232065308A0123206C3083
:102AC0008A01232065308A01232063308A01232074
:102AD00074308A01232020308A01232043308A0168
:102AE00023206F308A0123206D308A0123206D302E
:102AF0008A01232061308A0123206E308A0123203D
:102B000064308A01232020308A0123200A308A0180
:102B100023200D308A01232020308A0123204330D6
:102B20008A01232065308A0123206E308A01232008
:102B300074308A01232072308A01232065308A0193
:102B4000232020308A01232050308A012320753031
:102B50008A01232073308A01232068308A012320D0
:102B600020308A01232074308A0123206F308A01AB
:102B7000232020308A01232020308A012320533053
:102B80008A01232065308A0123206E308A012320A8
:102B900064308A01232020308A01232043308A01B7
:102BA00023206F308A0123206D308A0123206D306D
:102BB0008A01232061308A0123206E308A0123207C
:102BC00064308A01232021308A01232021308A01A8
:102BD00023200330A300E8308A01EB218A150A1272
:102BE0002D271B308A01232053308A0123200030F7
:102BF0008A01232007308A01232020308A012320E4
:102C000043308A0123206F308A0123206D308A01EE
:102C100023206D308A01232061308A0123206E3009
:102C20008A01232064308A01232020308A01232056
:102C300068088A01022020308A01232021308A017D
:102C4000232020308A0123200130A300F4308A01A0
:102C5000EB2164006908053C8A110A160319EE2D60
:102C600064006908003C8A110A16031D382EE80A20
:102C700064006908023C8A110A16031D402EE8030D
:102C800064006908043C8A110A16031DEE2D0A30FF
:102C90008A0123200A308A0123200D308A01232053
:102CA00043308A0123206F308A0123206E308A014D
:102CB000232066308A01232069308A012320723064
:102CC0008A0123206D308A01232020308A012320AD
:102CD00020308A01232028308A01232059308A019C
:102CE00023202F308A0123204E308A0123202930CF
:102CF0008A01232020308A0123203F308A012320AB
:102D000020308A01232055308A01232070308A0127
:102D100023203D308A01232059308A012320653049
:102D20008A01232073308A01232020308A01232046
:102D300044308A0123206F308A01232077308A01B2
:102D400023206E308A0123203D308A0123204E301B
:102D50008A0123206F308A0123200330A300E8304A
:102D60008A01EB218A150A122D2764006908003CAC
:102D70008A110A160319C62E64006908023C8A11DA
:102D80000A160319EC2F8A110A16B22E1B308A017B
:102D9000232043308A01232043308A0123206F30CF
:102DA0008A0123206D308A0123206D308A0123207F
:102DB00061308A0123206E308A01232064308A0129
:102DC000232020308A01232068088A010220203035
:102DD0008A01232053308A01232065308A01232071
:102DE0006E308A01232074308A0123206808A600EF
:102DF000A7011430A200A3018A016822EA00250875
:102E0000EB00061583160611033083128A01EA21AE
:102E1000061183160611013083128A01EA216A081D
:102E2000A0006B08A1000630840004308A01F42061
:102E30000130E4006400023064028A110A160318AB
:102E4000B42F0730B6008030B4000630B300E8304D
:102E5000B7000330B5008A0116218A150A16031C33
:102E60003028E900640068080C3C8A110A16031D2A
:102E7000682F0A308A0123200D308A012320533025
:102E80008A0123206C308A01232061308A012320AB
:102E900076308A01232065308A01232020308A0180
:102EA000232064088A01022020308A012320563022
:102EB0008A01232069088A01022020308A01232008
:102EC0000130A300F4308A01EB218A110A16AF2FDA
:102ED0006400680869028A110A160319AF2F0A30C4
:102EE0008A0123200D308A01232053308A012320B8
:102EF0006C308A01232061308A01232076308A01D8
:102F0000232065308A01232020308A012320640891
:102F10008A01022020308A01232045308A012320A3
:102F200072308A01232072308A0123206F308A0197
:102F3000232072308A01232021308A0123200614A5
:102F40008316061083120B30A300B8308A01EB21E0
:102F500006108316061083128A110A16EC2FE40A53
:102F60008A110A16031D1A2F0A308A0123200D30F8
:102F70008A01232041308A01232063308A012320E3
:102F80006B308A0123206E308A0123206F308A0142
:102F9000232077308A0123206C308A01232065307A
:102FA0008A01232064308A01232067308A0123208C
:102FB00065308A01232064308A01232020308A0171
:102FC00023204F308A0123204B308A0123200330F5
:102FD000A300E8308A01EB210A308A0123200D305A
:102FE0008A01232041308A0123206E308A01232068
:102FF00079308A01232020308A0123204B308A0136
:10300000232065308A01232079308A012320203053
:103010008A01232054308A0123206F308A01232023
:1030200020308A01232045308A01232078308A010C
:10303000232069308A01232074308A0123208A15D5
:103040000A122D2764006908053C8A150A1603191F
:103050001F281B308A0123205F308A0123200800AB
:103060000A308A0123200D308A0123202A308A0168
:10307000232020308A01232043308A0123206F300F
:103080008A0123206D308A0123206D308A0123209C
:1030900073308A01232020308A01232045308A01A1
:1030A000232072308A01232072308A0123206F305E
:1030B0008A01232072308A01232021308A012320B3
:1030C00020308A0123202A308A0123200614831607
:1030D000061083120B30A300B8308A01EB210610D2
:1030E0008316061083128A110A16EC2F0730B600D9
:1030F0000430B40001308A01D42033308A01BC206E
:103100008A01D1200730B6000430B40000308A01B3
:10311000D4200830A900A130B000B101A501383099
:103120008A018E218A01D1201B308A01232043305D
:103130008A01232046308A01232061308A0123201E
:103140006D308A01232069308A0123206C308A0186
:10315000232079308A01232020308A0123203D302A
:103160008A01232020308A0123200230A900380858
:10317000A400A5012230B000B1018A019E2168306F
:103180008A0123200A308A0123200A308A01232061
:103190000D308A0123200230A9003908A400A501BE
:1031A0002230B000B1018A019E2120308A01232003
:1031B0000230A9003A08A400A5012230B000B101F4
:1031C0008A019E2120308A0123200230A9003B0879
:1031D000A400A5012230B000B1018A019E2168300F
:1031E0008A0123200A308A0123200D308A012320FE
:1031F0000230A9003C08A400A5012230B000B101B2
:103200008A019E2120308A0123200230A9003D0836
:10321000A400A5012230B000B1018A019E21203016
:103220008A0123200230A9003E08A400A501223013
:10323000B000B1018A019E2168308A0123200A3042
:103240008A0123200A308A0123200D308A0123209D
:1032500043308A01232052308A01232043308A01DF
:10326000232020308A01232056308A012320613018
:103270008A0123206C308A01232020308A012320F8
:103280003D308A01232020308A0123200230A9000A
:103290003F08A400A5012230B000B1018A019E219F
:1032A00068308A0123200730A300D0308A01EB2147
:0632B0008A110A16EC2F42
:02400E00F42399
:00000001FF
